S123F8008E00FFCE10001F2E40FC8630A72B8600A72C860CA72D863CA7098650A728BDF8DD
S123F8206DBDF87EBDF886BDF88218CEF8DFBDF899BDF86D188CF8EB26F420EE1F2E20FC6D
S123F840A62F391F2E80FCA72F39183C18CE00181809188C000026F81838E608C4DFE708B9
S123F860A72A1F2980FCE608CA20E70839183C18CEC4001809188C000026F818383986639C
S123F8802006866220028661BDF84A8665BDF84A860FBDF84ABDF84A398661BDF84A8670BC
S123F8A0BDF84A8601BDF84A18A600BDF84A18088661BDF84A8670BDF84A8602BDF84A1868
S123F8C0A600BDF84A18088661BDF84A8670BDF84A8603BDF84A18A600BDF84A1808398363
S10FF8E0706D83C3C6DAC3C6D98C6D00FA
S105FFFEF80005
S9030000FC
